:020000020000FC
:0200000009C035
:100012008CC00FEE0ABB0FEE0BBB07E007BB00E084
:1000220008BB0FED0DBF00E808B900E205BF03E011
:1000320000B902E000BF03E003BF01EB06BF02E02C
:1000420009BF00E00FBD07E00EBD31E041E011271E
:100052002227FF24CC2778948895FECF0FEE0BBB86
:10006200E8E3F0E0042F0A95E00FFF1D099406C0B3
:1000720008C00AC00CC00EC010C012C058BBD8982D
:10008200089568BBD998089578BBDA98089588BB1B
:10009200DB98089598BBDD980895A8BBDE98089573
:1000A200B8BBDF9808950A3030F4F1E0E2E7E00FE0
:1000B200FF1D0491089507E708951CB52DB5133669
:1000C2002F0518F019E029E006C022271A3018F08F
:1000D2001A502395FBCF552766277727882799271C
:1000E200AA27BB27012FDFDF00FF51E001FF61E0FC
:1000F20002FF71E003FF81E004FF91E005FFA1E050
:1001020006FFB1E0203081F0022FCDDF00FF526008
:1001120001FF626002FF726003FF826004FF92606F
:1001220005FFA26006FFB26008954A95F9F447E020
:100132003A9569F439E1C13041F050E060E070E095
:1001420080E090E0A0E0B1E011C0B7DF0FC03C302A
:1001520069F4C0E009B304FFC1E0FDBCFCBC54601B
:100162006460746084609460A460B46077DF189502
:0A01720040792430191202780010C1
:00000001FF
